:020000040800F2
:1000000000060020E1010008410E0008C10D0008B3
:10001000190E0008C10D0008ED0D0008E3010008ED
:10002000E3010008E3010008E301000819210008CA
:10003000E3010008E3010008E3010008E301000810
:10004000E3010008E3010008E3010008E301000800
:10005000E3010008E3010008E13100080D32000867
:10006000393200086532000891320008E3010008C7
:10007000E3010008E3010008E3010008E3010008D0
:10008000E3010008E3010008E3010008E3010008C0
:10009000E3010008E3010008E3010008BD320008A5
:1000A000E3010008E3010008E3010008E3010008A0
:1000B00055300008E3010008E3010008E3010008EF
:1000C000E3010008E3010008E3010008E301000880
:1000D000E3010008E3010008E3010008E301000870
:1000E00025330008E3010008E3010008E3010008EC
:1000F000E3010008E3010008E3010008E301000850
:10010000E3010008E3010008E3010008E30100083F
:10011000E3010008E3010008E3010008E30100082F
:10012000E3010008E3010008E3010008E30100081F
:10013000E3010008E3010008E3010008E30100080F
:10014000E3010008E3010008E3010008512800086A
:10015000E3010008E3010008E3010008E3010008EF
:10016000E3010008E3010008E3010008E3010008DF
:10017000E3010008E3010008E3010008E3010008CF
:10018000E3010008E3010008E3010008E3010008BF
:10019000E3010008E3010008E3010008E3010008AF
:1001A000E3010008E3010008E3010008E30100089F
:1001B000E3010008E3010008E3010008E30100088F
:1001C000E3010008E3010008E3010008E30100087F
:1001D000E3010008E3010008E3010008E30100086F
:1001E00002E000F000F8FEE772B63A4880F30888B3
:1001F000394880F3098839484EF60851CEF200019B
:10020000086040F20000CCF200004EF63471CEF2ED
:1002100000010860BFF34F8FBFF36F8F40F2000003
:10022000C0F2F0004EF68851CEF200010860BFF334
:100230004F8FBFF36F8F4FF00000E1EE100A4EF6C4
:100240003C71CEF200010860062080F31488BFF3F1
:100250006F8F01F0E1FF01F0BDFF02F05FFE4FF094
:1002600055301F491B4A91423CBF41F8040BFAE745
:100270001C49194A91423CBF41F8040BFAE71A495C
:100280001A4A1B4B9A423EBF51F8040B42F8040B2A
:10029000F8E700201749184A91423CBF41F8040B87
:1002A000FAE701F09BFF02F08DFE144C144DAC42B6
:1002B00003DA54F8041B8847F9E700F041F8114CC1
:1002C000114DAC4203DA54F8041B8847F9E701F0FA
:1002D00083BF00000006002000220020000000086C
:1002E00000000020000600206837000800220020DF
:1002F0004022002040220020A82D0020E00100081C
:10030000E0010008E0010008E00100082DE9F04FDD
:100310002DED108AC1F80CD0C3689D46BDEC108A43
:10032000BDE8F08F002383F311882846A047002002
:1003300001F0FCFAFEE701F077FA00DFFEE70000CB
:1003400038B501F0B9FE054601F0DCFE0446D8B927
:100350000F4B9D421AD001339D4218BF044641F213
:10036000883504BF01240025002001F0AFFE0CB148
:1003700000F076F800F0FAFC00F0A0FB284600F050
:10038000BFF800F06DF8F9E70025EDE70546EBE76B
:10039000010007B008B500F063FBA0F1200358424C
:1003A000584108BD07B541F21203022101A8ADF87A
:1003B000043000F073FB03B05DF804FB38B5202374
:1003C00083F311881748C3680BB101F035FB164A57
:1003D000144800234FF47A7101F0F2FA002383F3FA
:1003E0001188124C236813B12368013B23606368B2
:1003F00013B16368013B63600D4D2B7833B96368BB
:100400007BB9022000F02CFC322363602B78032B95
:1004100007D163682BB9022000F022FC4FF47A73F5
:10042000636038BD40220020BD0300085C2300202B
:1004300054220020084B187003280CD8DFE800F085
:1004400008050208022000F001BC022000F0F4BB05
:10045000024B00225A607047542200205C23002087
:10046000234B244A10B51C46196801313FD0043390
:100470009342F9D16268A24239D31F4B9B6803F1C2
:10048000006303F540439A4231D2002000F030FB74
:100490000220FFF7CFFF194B1A6C00221A64196E65
:1004A0001A66196E596C5A64596E5A665A6E5A69B0
:1004B00042F080025A615A6922F080025A615A69F8
:1004C0001A6942F000521A611A6922F000521A6148
:1004D0001B6972B64FF0E0232021C3F8084DD4E920
:1004E000003281F311889D4683F30888104710BDC0
:1004F00000C0000820C00008002200200038024090
:100500002DE9F04F93B0AA4B00902022FF210AA8BA
:100510009D6800F0D5FBA74A1378A3B9A64801212E
:10052000C3601170202383F31188C3680BB101F0FD
:1005300083FAA24AA04800234FF47A7101F040FAEE
:10054000002383F31188009B13B19D4B009A1A601E
:100550009C4A009C1378032B1EBF00231370984AFB
:100560004FF0000A18BF5360D3465646D1460120CB
:1005700000F06CFB24B1924B1B68002B00F0118241
:10058000002000F06DFA0390039B002BF2DB0120AA
:1005900000F052FB039B213B162BE8D801A252F836
:1005A00023F000BF0106000829060008BD06000868
:1005B0006F0500086F0500086F0500084707000871
:1005C000170900083108000893080008BB08000854
:1005D000E10800086F050008F30800086F0500082F
:1005E00065090008A10600086F050008A9090008B0
:1005F0000D060008A10600086F0500089308000812
:100600000220FFF7C7FE002840F0F581009B022181
:10061000BAF1000F08BF1C4605A841F21233ADF82D
:10062000143000F03BFAA2E74FF47A7000F018FAA9
:10063000071EEBDB0220FFF7ADFE0028E6D0013FEE
:10064000052F00F2DA81DFE807F0030A0D101336F8
:1006500005230593042105A800F020FA17E054486B
:100660000421F9E758480421F6E758480421F3E744
:100670004FF01C08404600F03DFA08F104080590D0
:10068000042105A800F00AFAB8F12C0FF2D10120DC
:1006900000FA07F747EA0B0B5FFA8BFB4FF00009F4
:1006A00000F05AFB26B10BF00B030B2B08BF002404
:1006B000FFF778FE5BE746480421CDE7002EA5D082
:1006C0000BF00B030B2BA1D10220FFF763FE0746B3
:1006D00000289BD0012000F00BFA0220FFF7AAFEB1
:1006E00000265FFA86F8404600F012FA044690B100
:1006F0000021404600F01CFA01360028F1D1BA462C
:10070000044641F21213022105A8ADF814303E460A
:1007100000F0C4F92BE70120FFF78CFE2546244B9F
:100720009B68AB4207D9284600F0E4F9013040F05D
:1007300067810435F3E7234B00251D70204BBA4633
:100740005D603E46ACE7002E3FF460AF0BF00B035C
:100750000B2B7FF45BAF0220FFF76CFE322000F022
:100760007FF9B0F10008FFF651AF18F003077FF4EE
:100770004DAF0F4A926808EB050393423FF646AF30
:10078000B8F5807F3FF742AF124B0193B84523DDA8
:100790004FF47A7000F064F90390039A002AFFF690
:1007A00035AF019B039A03F8012B0137EDE700BF3A
:1007B000002200205823002040220020BD03000812
:1007C0005C23002054220020042200200822002064
:1007D0000C22002058220020C820FFF7DBFD07462E
:1007E00000283FF413AF1F2D11D8C5F12002424558
:1007F0000AAB25F0030028BF424683490192184402
:1008000000F038FA019A8048FF2100F059FA4FEAC7
:10081000A8037D490193C8F38702284600F058FADF
:10082000064600283FF46DAF019B05EB830537E7D3
:100830000220FFF7AFFD00283FF4E8AE00F0A4F976
:1008400000283FF4E3AE0027B846704B9B68BB42DC
:1008500018D91F2F11D80A9B01330ED027F003039C
:1008600012AA134453F8203C05934046042205A9DC
:1008700000F0E8FA04378046E7E7384600F03AF936
:100880000590F2E7CDF81480042105A800F006F9E0
:1008900006E70023642104A8049300F0F5F800287B
:1008A0007FF4B4AE0220FFF775FD00283FF4AEAE32
:1008B000049800F051F90590E6E70023642104A8AC
:1008C000049300F0E1F800287FF4A0AE0220FFF7C7
:1008D00061FD00283FF49AAE049800F04DF9EAE774
:1008E0000220FFF757FD00283FF490AE00F05CF9BE
:1008F000E1E70220FFF74EFD00283FF487AE05A98F
:10090000142000F057F904210746049004A800F0D1
:10091000C5F83946B9E7322000F0A2F8071EFFF605
:1009200075AEBB077FF472AE384A926807EB0903D5
:1009300093423FF66BAE0220FFF72CFD00283FF4F8
:1009400065AE27F003074F44B9453FF4A9AE4846CA
:1009500000F0D0F80421059005A800F09FF809F1F7
:100960000409F1E74FF47A70FFF714FD00283FF413
:100970004DAE00F009F9002844D00A9B01330BD09A
:1009800008220AA9002000F0A3F900283AD020226A
:10099000FF210AA800F094F9FFF704FD1C4800F0BD
:1009A000CBFF13B0BDE8F08F002E3FF42FAE0BF05D
:1009B0000B030B2B7FF42AAE0023642105A80593BB
:1009C00000F062F8074600287FF420AE0220FFF70F
:1009D000E1FC804600283FF419AEFFF7E3FC41F24A
:1009E000883000F0A9FF059800F0E8F9464600F0CD
:1009F000B3F93C46BBE5064652E64FF0000905E672
:100A0000BA467EE637467CE65822002000220020C7
:100A1000A086010070B50F4B1B780133DBB2012BB0
:100A20000C4611D80C4D29684FF47A730E6AA2FB5C
:100A30000332014622462846B047844204D1074B80
:100A400000221A70012070BD4FF4FA7000F074FF9C
:100A50000020F8E7102200205025002090230020DD
:100A600007B50023024601210DF107008DF807307C
:100A7000FFF7D0FF20B19DF8070003B05DF804FB3D
:100A80004FF0FF30F9E700000A4608B50421FFF7F0
:100A9000C1FF80F00100C0B2404208BD30B4054C37
:100AA0002368DD69044B0A46AC460146204630BC4B
:100AB000604700BF50250020A086010070B501F0FE
:100AC000EDF9094E094D30800024286833888342AF
:100AD00008D901F0DDF92B6804440133B4F5404F27
:100AE0002B60F2D370BD00BF92230020642300204E
:100AF00001F096BA00F1006000F5404000687047D0
:100B000000F10060920000F5404001F015BA0000CD
:100B1000054B1A68054B1B889B1A834202D9104467
:100B200001F0B6B900207047642300209223002012
:100B300038B5084D044629B128682044BDE838403E
:100B400001F0C6B92868204401F0AAF90028F3D0C2
:100B500038BD00BF6423002010F003030AD1B0F5B4
:100B6000047F05D200F10050A0F51040D0F8003805
:100B7000184670470023FBE700F10050A0F5104035
:100B8000D0F8100A70470000064991F8243033B1BC
:100B90000023086A81F824300822FFF7B1BF012042
:100BA000704700BF68230020014B1868704700BFE2
:100BB000002004E0F0B51C4B024618681B4BC0F344
:100BC0000B050424000C1E88AE421BD15C6893F90F
:100BD0000850174B05261F88874208BF93F902501B
:100BE000013E03F10403F6D1013A0A44013C0B46ED
:100BF00093420ED214F9016F581C66B100F8016CD3
:100C00000346F5E7013C03F10C03DCD1094C3F2519
:100C1000DFE7184605E02C2490421C7001D2981C96
:100C20005D70401AF0BD00BF002004E0643400088D
:100C30005034000824340008022802BF024B4FF051
:100C400000729A61704700BF00000240022802BF94
:100C5000024B4FF400729A61704700BF00000240DF
:100C6000022801BF024A536983F40073536170473D
:100C70000000024010B50023934203D0CC5CC45462
:100C80000133F9E710BD000010B5013810F9013F3C
:100C90003BB191F900409C4203D11AB10131013AB4
:100CA000F4E71AB191F90020981A10BD1046FCE73C
:100CB00003460246D01A12F9011B0029FAD17047E7
:100CC00002440346934202D003F8011BFAE770473F
:100CD0002DE9F8431F4D144695F824200746884611
:100CE00052BBDFF870909CB395F824302BB92022CA
:100CF000FF2148462F62FFF7E3FF95F82400C0F17B
:100D00000802A24228BF2246D6B24146920005EB15
:100D10008000FFF7AFFF95F82430A41B1E44F6B205
:100D2000082E17449044E4B285F82460DBD1FFF725
:100D30002BFF0028D7D108E02B6A03EB8203834204
:100D4000CFD0FFF721FF0028CBD10020BDE8F883EA
:100D50000120FBE768230020024B1A78024B1A702F
:100D6000704700BF902300201022002010B50F4CC8
:100D70000F4800F0F7F821460D4800F01FF92468ED
:100D80000C48626DD2F8043843F00203C2F804380C
:100D900000F0D2FD0849204600F016FA626DD2F844
:100DA000043823F00203C2F8043810BD5835000897
:100DB0005025002040420F006035000870470000B9
:100DC00000B59BB0EFF3098168226846FFF752FF38
:100DD000EFF30583044B9A6BDA6A9A6A9A6A9A6A05
:100DE0009A6A9A6A9B6AFEE700ED00E000B59BB044
:100DF000EFF3098168226846FFF73CFFEFF30583B4
:100E0000044B9A6B9A6A9A6A9A6A9A6A9A6A9B6A75
:100E1000FEE700BF00ED00E000B59BB0EFF30981F5
:100E200068226846FFF726FFEFF30583034B5A6BF2
:100E30009A6A9A6A9A6A9A6A9B6AFEE700ED00E0EB
:100E4000FEE7000030B5094D0A4491420DD011F87B
:100E5000013B5840082340F30004013B2C4013F0B1
:100E6000FF0384EA5000F6D1EFE730BD2083B8EDF0
:100E7000026843681143016003B1184770470000DE
:100E800013B5446BD4F894341A681178042915D139
:100E9000217C022912D11979128901238B40134236
:100EA0000CD101A904F14C0001F03EFFD4F89444A8
:100EB000019B21790246206800F0CEF902B010BDF6
:100EC000143001F0C1BE00004FF0FF33143001F0C8
:100ED000BBBE00004C3001F093BF00004FF0FF3369
:100EE0004C3001F08DBF0000143001F08FBE0000C7
:100EF0004FF0FF31143001F089BE00004C3001F09A
:100F00005FBF00004FF0FF324C3001F059BF0000CE
:100F10000020704710B5D0F894341A68117804296D
:100F2000044617D1017C022914D159795289012331
:100F30008B4013420ED1143001F022FE024648B11C
:100F4000D4F894444FF4807361792068BDE8104070
:100F500000F070B910BD0000406BFFF7DBBF000070
:100F6000704700007FB5124B036000234360C0E967
:100F70000233012502260F4B0574044602900193AB
:100F800000F18402294600964FF48073143001F07A
:100F9000D3FD094B0294CDE9006304F523724FF4AD
:100FA0008073294604F14C0001F09AFE04B070BD34
:100FB00094340008590F0008810E00080B682022A5
:100FC00082F311880A7903EB820290614A7909322F
:100FD00043F822008A7912B103EB8203986102235D
:100FE0000374C0F89414002383F311887047000041
:100FF00038B5037F044613B190F85430ABB9201DC7
:1010000001250221FFF734FF04F1140025776FF06A
:10101000010100F0B9FC84F8545004F14C006FF069
:101020000101BDE8384000F0AFBC38BD10B501216A
:1010300004460430FFF71CFF0023237784F8543064
:1010400010BD000038B504460025143001F08CFDB9
:1010500004F14C00257701F05BFE201D84F854500C
:101060000121FFF705FF2046BDE83840FFF752BFDA
:1010700090F8443003F06003202B07D190F845200E
:10108000212A4FF0000303D81F2A06D800207047FA
:10109000222AFBD1C0E90E3303E0034A8263072210
:1010A000C2630364012070471122002037B5D0F8D5
:1010B00094341A681178042904461AD1017C022953
:1010C00017D11979128901238B40134211D100F1F4
:1010D0004C05284601F0DCFE58B101A9284601F074
:1010E00023FED4F89444019B21790246206800F045
:1010F000B3F803B030BD0000F0B500EB810385B05C
:101100009E6904460D46FEB1202383F3118804EB4B
:101110008507301D0821FFF7ABFEFB685B691B6884
:1011200006F14C001BB1019001F00CFE019803A9DF
:1011300001F0FAFD024648B1039B2946204600F023
:101140008BF8002383F3118805B0F0BDFB685A6962
:101150001268002AF5D01B8A013B1340F1D104F13B
:101160004402EAE7093138B550F82140DCB12023C8
:1011700083F31188D4F894241368527903EB820323
:10118000DB689B695D6845B104216018FFF770FE5C
:10119000294604F1140001F0FDFC2046FFF7BAFED9
:1011A000002383F3118838BD7047000001F0AAB80E
:1011B000012303700023C0E90133C361836203622A
:1011C000C36243620363704738B50446202383F348
:1011D00011880025C0E90355C0E90555416001F0BB
:1011E000A1F80223237085F3118838BD70B500EB98
:1011F000810305465069DA600E46144618B1102284
:101200000021FFF75DFDA06918B110220021FFF752
:1012100057FD31462846BDE8704001F04DB9000049
:10122000826802F0011282600022C0E90422826119
:1012300001F0CEB9F0B400EB81044789E4680125E0
:10124000A4698D403D43458123600023A260636013
:10125000F0BC01F0E9B90000F0B400EB81040789AB
:10126000E468012564698D403D43058123600023C6
:10127000A2606360F0BC01F063BA000070B50223A5
:10128000002504460370C0E90255C0E90455C56451
:10129000856180F8345001F0ABF863681B6823B1B6
:1012A00029462046BDE87040184770BD037880F895
:1012B00050300523037043681B6810B504460BB11A
:1012C000042198470023A36010BD000090F850202F
:1012D000436802701B680BB1052118477047000076
:1012E00070B590F83430044613B1002380F83430E0
:1012F00004F14402204601F08DF963689B68B3B99C
:1013000094F8443013F0600535D00021204601F0F8
:10131000DFFB0021204601F0D1FB63681B6813B19D
:10132000062120469847062384F8343070BD2046B5
:1013300098470028E4D0B4F84A30E26B9A4288BF5C
:10134000E36394F94430E56B002B4FF0200380F207
:101350000381002D00F0F280092284F8342083F309
:1013600011880021D4E90E232046FFF775FF0023E2
:1013700083F31188DAE794F8452003F07F0343EA0A
:10138000022340F20232934200F0C58021D8B3F527
:10139000807F48D00DD8012B3FD0022B00F09380E6
:1013A000002BB2D104F14C02A2630222E263236457
:1013B000C1E7B3F5817F00F09B80B3F5407FA4D1F6
:1013C00094F84630012BA0D1B4F84C3043F002031E
:1013D00032E0B3F5006F4DD017D8B3F5A06F31D020
:1013E000A3F5C063012B90D8636894F846205E682B
:1013F00094F84710B4F848302046B047002884D00D
:101400004368A3630368E3631AE0B3F5106F36D053
:1014100040F6024293427FF478AF5C4BA363022311
:10142000E3630023C3E794F84630012B7FF46DAFEC
:10143000B4F84C3023F00203C4E90E55A4F84C3044
:10144000256478E7B4F84430B3F5A06F0ED194F872
:10145000463084F84E30204601F022F863681B685D
:1014600013B1012120469847032323700023C4E9C8
:101470000E339CE704F14F03A3630123C3E72378F2
:10148000042B10D1202383F311882046FFF7C8FED8
:1014900085F311880321636884F84F5021701B681D
:1014A0000BB12046984794F84630002BDED084F8E4
:1014B0004F300423237063681B68002BD6D00221B1
:1014C00020469847D2E794F848301D0603F00F01F4
:1014D00020460AD501F090F8012804D002287FF4B4
:1014E00014AF2B4B9AE72B4B98E701F077F8F3E713
:1014F00094F84630002B7FF408AF94F8483013F08E
:101500000F01B3D01A06204602D501F0F5FAADE777
:1015100001F0E8FAAAE794F84630002B7FF4F5AE24
:1015200094F8483013F00F01A0D01B06204602D5D6
:1015300001F0CEFA9AE701F0C1FA97E7142284F895
:10154000342083F311882B462A4629462046FFF78C
:1015500071FE85F31188E9E65DB1152284F8342027
:1015600083F311880021D4E90E232046FFF762FEA1
:10157000FDE60B2284F8342083F311882B462A469B
:1015800029462046FFF768FEE3E700BFC4340008A1
:10159000BC340008C034000838B590F83430044634
:1015A000002B3ED0063BDAB20F2A34D80F2B32D8AC
:1015B000DFE803F037313108223231313131313156
:1015C00031313737C56BB0F84A309D4214D2C36809
:1015D0001B8AB5FBF3F203FB12556DB9202383F38D
:1015E00011882B462A462946FFF736FE85F31188D7
:1015F0000A2384F834300EE0142384F83430202396
:1016000083F3118800231A4619462046FFF712FE7D
:10161000002383F3118838BD036C03B1984700237E
:10162000E7E70021204601F053FA0021204601F0AF
:1016300045FA63681B6813B10621204698470623C4
:10164000D7E7000010B590F83430142B044629D0A9
:1016500017D8062B05D001D81BB110BD093B022BB2
:10166000FBD80021204601F033FA0021204601F08A
:1016700025FA63681B6813B10621204698470623A4
:1016800019E0152BE9D10B2380F83430202383F3A4
:10169000118800231A461946FFF7DEFD002383F365
:1016A0001188DAE7C3689B695B68002BD5D1036CAE
:1016B00003B19847002384F83430CEE7024B002270
:1016C000C3E900339A607047942300200023037419
:1016D0008268054B1B6899689142FBD25A68036087
:1016E00042601060586070479423002008B52023A2
:1016F00083F31188037C032B05D0042B0DD02BB969
:1017000083F3118808BD436900221A604FF0FF334C
:101710004361FFF7DBFF0023F2E7D0E900321360FB
:101720005A60F3E7002303748268054B1B689968CD
:101730009142FBD85A68036042601060586070475D
:1017400094230020054B19690874186802681A6010
:101750005360186101230374FEF7D8BD9423002061
:1017600030B54B1C0B4D87B0044610D02B690A4A8C
:1017700001A800F025F92046FFF7E4FF049B13B110
:1017800001A800F059F92B69586907B030BDFFF77F
:10179000D9FFF8E794230020ED16000838B50C4D6A
:1017A00041612B6981689A689142044603D8BDE87B
:1017B0003840FFF78BBF1846FFF7B4FF01232C61B9
:1017C000014623742046BDE83840FEF79FBD00BFA8
:1017D00094230020044B1A681B6990689B68984208
:1017E00094BF0020012070479423002010B5084CBE
:1017F000236820691A6822605460012223611A74E8
:10180000FFF790FF01462069BDE81040FEF77EBD5E
:101810009423002008B5FFF7DDFF18B1BDE80840AC
:10182000FFF7E4BF08BD0000FFF7E0BFFEE70000E0
:1018300010B50C4CFFF742FF00F0B4F80A498022C3
:10184000204600F03BF8012344F8180C037400F024
:1018500073FC002383F3118862B60448BDE810408E
:1018600000F04CB8BC230020C8340008D83400086D
:1018700000F01CB9EFF3118020B9EFF305832022AB
:1018800082F311887047000010B530B9EFF305847A
:10189000C4F3080414B180F3118810BDFFF7BAFF38
:1018A00084F31188F9E70000034A516853685B1A12
:1018B0009842FBD8704700BF001000E0826002220F
:1018C000028270478368A3F17C0243F80C2C026902
:1018D00043F83C2C426943F8382C074A43F81C2C47
:1018E000C26843F8102C022203F8082C002203F8E7
:1018F000072CA3F1180070472503000810B520231A
:1019000083F31188FFF7DEFF00210446FFF746FF4F
:10191000002383F31188204610BD0000024B1B6991
:1019200058610F20FFF70EBF94230020202383F37C
:101930001188FFF7F3BF000008B50146202383F3A9
:1019400011880820FFF70CFF002383F3118808BDDE
:1019500049B1064B42681B6918605A6013604360C6
:101960000420FFF7FDBE4FF0FF30704794230020A6
:101970000368984206D01A680260506059611846A0
:10198000FFF7A4BE7047000038B504460D46206836
:10199000844200D138BD036823605C604561FFF775
:1019A00095FEF4E7054B03F11402C3E905224FF05D
:1019B000FF310022C3E90712704700BF94230020C3
:1019C00070B51C4EC0E9032305460C4601F092FA9F
:1019D000334653F8142F9A420DD13062C5E90124E1
:1019E0002A600A2C2CBF00190A30C6E90555BDE84B
:1019F000704001F06DBA316A431AE31838BF1C46D3
:101A00009368A34202D9081901F070FA73699A68C1
:101A100094420CD85A68AC602B606A6015609A6872
:101A20005D60121B9A604FF0FF33F36170BD1B685D
:101A3000A41AECE79423002038B51B4C6369984244
:101A40000DD0D0E9003213605A6000228168C26074
:101A50009A680A449A604FF0FF33E36138BD22462A
:101A6000036842F8143F002193425A60C16003D1D9
:101A7000BDE8384001F034BA9A688168256A0A44A2
:101A80009A6001F037FA63699A68411B8A42E5D986
:101A9000AB181D1A092D206A98BF01F10A02BDE892
:101AA0003840104401F022BA942300202DE9F0417F
:101AB000184C002704F11406656901F01BFA236A2B
:101AC000AA68C11A8A4215D813442362D5E90032A4
:101AD00013605A606369D5F80C80EF60B34201D19E
:101AE00001F0FEF987F311882869C047202383F3AA
:101AF0001188E1E76169B14209D013441B1ABDE8BE
:101B0000F0410A2B2CBFC0180A3001F0EFB9BDE834
:101B1000F08100BF9423002000207047FEE7000002
:101B2000704700004FF0FF307047000002290CD0D2
:101B3000032904D00129074818BF00207047032A51
:101B400005D8054800EBC2007047044870470020E4
:101B5000704700BFBC350008202200207035000807
:101B600070B59AB00546084601A9144600F0C2F8BF
:101B700001A8FFF79DF8431C5B00C5E90034002273
:101B8000237003236370C6B201AB02341046D1B296
:101B90008E4204F1020401D81AB070BD13F8011B83
:101BA00004F8021C04F8010C0132F0E708B5202308
:101BB00083F311880348FFF779FA002383F3118830
:101BC00008BD00BF5025002090F8443003F01F02EC
:101BD000012A07D190F845200B2A03D10023C0E940
:101BE0000E3315E003F06003202B08D1B0F8483025
:101BF0002BB990F84520212A03D81F2A04D8FFF7D3
:101C000037BA222AEBD0FAE7034A82630722C2637B
:101C100003640120704700BF1822002007B5052982
:101C200017D8DFE801F0191603191920202383F3D0
:101C30001188104A01900121FFF7D8FA01980E4A45
:101C40000221FFF7D3FA0D48FFF7FCF9002383F3D5
:101C5000118803B05DF804FB202383F31188074843
:101C6000FFF7C6F9F2E7202383F311880348FFF753
:101C7000DDF9EBE710350008343500085025002069
:101C800038B50C4D0C4C0D492A4604F10800FFF7FD
:101C900067FF05F1CA0204F110000949FFF760FF70
:101CA00005F5CA7204F118000649BDE83840FFF78F
:101CB00057BF00BF182A002020220020F03400085F
:101CC000FA3400080535000870B5044608460D468C
:101CD000FEF7EEFFC6B22046013403780BB9184672
:101CE00070BD32462946FEF7CFFF0028F3D1012010
:101CF000F6E700002DE9F04705460C46FEF7D8FF51
:101D00002C49C6B22846FFF7DFFF08B10836F6B205
:101D100029492846FFF7D8FF08B11036F6B2632EDE
:101D20000BD8DFF89080DFF89090244FDFF898A070
:101D30002E7846B92670BDE8F08729462046BDE8D2
:101D4000F04701F067BB252E30D1072241462846D7
:101D5000FEF79AFF80B91A4B224603F10C0153F8A3
:101D6000040B42F8040B8B42F9D119889B7811803F
:101D7000937007350F34DBE7082249462846FEF703
:101D800083FF98B90F4BA21C197809090232C95D6B
:101D900002F8041C13F8011B01F00F015345C95D43
:101DA00002F8031CF0D118340835C1E704F8016BC0
:101DB0000135BDE7DC35000805350008F4350008BD
:101DC000E4350008107AFF1F1C7AFF1FBFF34F8F06
:101DD000024AD368DB03FCD4704700BF003C0240DA
:101DE00008B5094B1B7873B9FFF7F0FF074B1A6969
:101DF000002ABFBF064A5A6002F188325A601A6848
:101E000022F480621A6008BD762C0020003C02405B
:101E10002301674508B50B4B1B7893B9FFF7D6FF35
:101E2000094B1A6942F000421A611A6842F4805262
:101E30001A601A6822F480521A601A6842F48062AA
:101E40001A6008BD762C0020003C02400B28F0B53B
:101E500016D80C4C0C4923787BB90C4D0E460C233C
:101E60004FF0006255F8047B46F8042B013B13F059
:101E7000FF033A44F6D10123237051F82000F0BD4E
:101E80000020FCE7A82C0020782C00200836000851
:101E9000014B53F820007047083600080C207047AB
:101EA0000B2810B5044601D9002010BDFFF7CEFF66
:101EB000064B53F824301844C21A0BB90120F4E73A
:101EC00012680132F0D1043BF6E700BF0836000883
:101ED0000B2838B5044628D8FFF7CCFCFFF776FF6F
:101EE000FFF77EFF124AF323D360E300DBB243F433
:101EF000007343F002031361136943F480331361E9
:101F000005462046FFF762FFFFF7A0FF094B53F895
:101F1000241000F0E9F82846FFF77CFFFFF7B4FC37
:101F20002046BDE83840FFF7BBBF002038BD00BFEA
:101F3000003C02400836000812F001032DE9F04190
:101F400005460E4614464BD18218B2F1016F61D896
:101F5000314B1B6813F001035CD0304FFFF78AFC54
:101F6000FFF73EFFF323FB60FFF730FF314640F2FF
:101F70000128032C18D824F00104284E0C446D1AB3
:101F800040F20118A142336905EB01072AD123F081
:101F900001033361FFF73EFFFFF776FC0120BDE848
:101FA000F081043C0435E4E7AB07E4D13B6923F45A
:101FB00040733B613B6943EA08033B6151F8046BA2
:101FC0002E60BFF34F8FFFF701FF2B689E42E8D0D2
:101FD0003B6923F001033B61FFF71CFFFFF754FC53
:101FE0000020DCE723F440733361336943EA0803DC
:101FF00033610B883B80BFF34F8FFFF7E7FE3F88CD
:1020000031F8023BBFB2BB42BCD0336923F00103BD
:102010003361E1E71846C2E700380240003C024065
:10202000084908B50B7828B11BB9FFF7D9FE012381
:102030000B7008BD002BFCD0BDE808400870FFF70E
:10204000E9BE00BF762C002010B50244064BD2B288
:10205000904200D110BD441C00B253F8200041F85A
:10206000040BE0B2F4E700BF502800400F4B30B53E
:102070001C6F240407D41C6F44F400741C671C6F8D
:1020800044F400441C670A4C236843F480732360C3
:102090000244084BD2B2904200D130BD441C00B281
:1020A00051F8045B43F82050E0B2F4E700380240F6
:1020B000007000405028004007B5012201A900200F
:1020C000FFF7C2FF019803B05DF804FB13B50446A7
:1020D000FFF7F2FFA04205D0012201A900200194E0
:1020E000FFF7C4FF02B010BD70470000034B1A6831
:1020F0001AB9034AD2F874281A607047AC2C002031
:102100000030024008B5FFF7F1FF024B1868C0F33A
:10211000407008BDAC2C0020EFF3098305494A6BE1
:1021200022F001024A63683383F30988002383F3B2
:102130001188704700EF00E0202080F3118862B61C
:102140000C4B0D4AD96821F4E0610904090C0A43DB
:10215000DA60D3F8FC20094942F08072C3F8FC2011
:102160000A6842F001020A601022DA7783F822003E
:10217000704700BF00ED00E00003FA05001000E02A
:1021800010B5202383F311880E4B5B6813F40063B2
:1021900014D0F1EE103AEFF30984683C4FF08073ED
:1021A000E361094BDB6B236684F30988FFF712FBBD
:1021B00010B1064BA36110BD054BFBE783F31188FB
:1021C000F9E700BF00ED00E000EF00E03703000892
:1021D0003A03000870470000FEE700000A4B0B4876
:1021E0000B4A90420BD30B4BDA1C121AC11E22F081
:1021F00003028B4238BF00220021FEF761BD53F875
:10220000041B40F8041BECE7A8370008A82D0020A9
:10221000A82D0020A82D00207047000070B5D0E93F
:1022200015439E6800224FF0FF3504EB4213510125
:10223000D3F800090028BEBFD3F8000940F0804061
:10224000C3F80009D3F8000B0028BEBFD3F8000B79
:1022500040F08040C3F8000B013263189642C3F887
:102260000859C3F8085BE0D24FF00113C4F81C38DA
:1022700070BD00001D4B03EB80022DE9F043D2F846
:102280000CC05D6DDCF81420461CD2F800E005EBB4
:10229000063605EB4018516871450AD3D5F8343835
:1022A000012202FA00F023EA0000C5F83408BDE874
:1022B000F083BCF81040AEEB0103A34228BF2346D5
:1022C000D8F81849A4B2B3EB840FF0D89468A4F1FD
:1022D000040959F8047F3760A4EB09071F44042F51
:1022E000F7D81C440B4494605360D4E7B02C002012
:1022F000890141F02001016103699B06FCD4122091
:10230000FFF7D2BA10B5054C2046FEF751FF4FF04B
:10231000A0436365024BA36510BD00BFB02C002035
:102320005C36000870B50378012B054650D12A4B66
:10233000446D98421BD1294B5A6B42F080025A637C
:102340005A6D42F080025A655A6D5A6942F0800215
:102350005A615A6922F080025A610E2143205B695A
:1023600000F0D4FB1E4BE3601E4BC4F80038002382
:10237000C4F8003EC02323606E6D4FF40413A363C2
:102380003369002BFCDA012333610C20FFF78CFA50
:102390003369DB07FCD41220FFF786FA3369002B80
:1023A000FCDA0026A6602846FFF738FF6B68C4F801
:1023B0001068DB68C4F81468C4F81C684BB90A4B91
:1023C000A3614FF0FF336361A36843F00103A3608F
:1023D00070BD064BF4E700BFB02C0020003802406F
:1023E0004014004003002002003C30C0083C30C0D4
:1023F000F8B5446D054600212046FFF779FFA96D29
:1024000000234FF001128F68C4F834384FF0006693
:10241000C4F81C284FF0FF3004EB431201339F42F5
:10242000C2F80069C2F8006BC2F80809C2F8080BCC
:10243000F2D20B686A6DEB65636210231361166953
:1024400016F01006FBD11220FFF72EFAD4F8003850
:1024500023F4FE63C4F80038A36943F4402343F037
:102460001003A3610923C4F81038C4F814380A4BC8
:10247000EB604FF0C043C4F8103B084BC4F8003B7E
:10248000C4F81069C4F80039EB6D03F1100243F48D
:102490008013EA65A362F8BD38360008408000105A
:1024A000426D90F84E10D2F8003823F4FE6343EAF0
:1024B0000113C2F8003870472DE9F84300EB81039F
:1024C000456DDA68166806F00306731E022B05EBED
:1024D00041130C4680460FFA81F94FEA41104FF044
:1024E0000001C3F8101B4FF0010104F1100398BF65
:1024F000B60401FA03F391698EBF334E06F180569C
:1025000006F5004600293AD0578A04F158014901DE
:1025100037436F50D5F81C180B43C5F81C382B18DF
:102520000021C3F8101953690127611EA7409BB30E
:10253000138A928B9B08012A88BF5343D8F85C20EA
:10254000981842EA034301F1400205EB8202C8F801
:102550005C00214653602846FFF7CAFE08EB89005D
:10256000C3681B8A43EA8453483464011E432E51D6
:10257000D5F81C381F43C5F81C78BDE8F88305EB77
:102580004917D7F8001B21F40041C7F8001BD5F804
:102590001C1821EA0303C0E704F13F0305EB8303A2
:1025A0000A4A5A6028462146FFF7A2FE05EB491069
:1025B000D0F8003923F40043C0F80039D5F81C38AE
:1025C00023EA0707D7E700BF0080001000040002DD
:1025D000826D1268C265FFF721BE00005831436D5D
:1025E00049015B5813F4004004D013F4001F0CBFE2
:1025F00002200120704700004831436D49015B58BB
:1026000013F4004004D013F4001F0CBF022001207B
:102610007047000000EB8101CB68196A0B681360FA
:102620004B6853607047000000EB810330B5DD68F4
:10263000AA691368D36019B9402B84BF4023136083
:102640006B8A1468426D1C44013CB4FBF3F4634391
:10265000033323F0030302EB411043EAC44343F086
:10266000C043C0F8103B2B6803F00303012B09B2F1
:102670000ED1D2F8083802EB411013F4807FD0F865
:10268000003B14BF43F0805343F00053C0F8003BBD
:1026900002EB4112D2F8003B43F00443C2F8003B86
:1026A00030BD00002DE9F041244D6E6D06EB401366
:1026B0000446D3F8087BC3F8087B38070AD5D6F858
:1026C0001438190706D505EB84032146DB68284634
:1026D0005B689847FA071FD5D6F81438DB071BD577
:1026E00005EB8403D968CCB98B69488A5A68B2FB78
:1026F000F0F600FB16228AB91868DA6890420DD20B
:10270000121AC3E90024202383F311880B482146C1
:10271000FFF78AFF84F31188BDE8F081012303FAF3
:1027200004F26B8923EA02036B81CB68002BF3D0A0
:1027300021460248BDE8F041184700BFB02C0020F8
:1027400000EB810370B5DD68436D6C692668E66057
:102750004A0156BB1A444FF40020C2F810092A68F7
:1027600002F00302012A0AB20ED1D3F8080803EBE3
:10277000421410F4807FD4F8000914BF40F0805058
:1027800040F00050C4F8000903EB4212D2F80009EF
:1027900040F00440C2F80009D3F83408012202FADC
:1027A00001F10143C3F8341870BD19B9402E84BF3C
:1027B0004020206020682E8A8419013CB4FBF6F486
:1027C00040EAC44040F000501A44C6E7F8B5044659
:1027D0001E48456D05EB4413D3F80869C3F8086932
:1027E000F10717D5D5F81038DA0713D500EB8403B5
:1027F000D9684B691F68DA68974218D2D21B002744
:102800001A605F60202383F311882146FFF798FF49
:1028100087F31188330617D5D5F834280123A34050
:10282000134211D02046BDE8F840FFF723BD012335
:1028300003FA04F2038923EA020303818B68002B65
:10284000E8D021469847E5E7F8BD00BFB02C00204E
:102850002DE9F74F984C666D7569B3691D4015F405
:102860008058756107D02046FEF708FD03B0BDE82B
:10287000F04FFFF785BC002D12DAD6F8003E8E48E7
:102880009F071EBFD6F8003E23F00303C6F8003EA4
:10289000D6F8043823F00103C6F80438FEF716FD15
:1028A000280505D58448FFF7B9FC8348FEF7FEFCF0
:1028B000A9040CD5D6F8083813F0060FF36823F4F2
:1028C00070530CBF43F4105343F4A053F3602A0732
:1028D00004D56368DB680BB177489847EB0274D482
:1028E000AF0227D5D4F85490DFF8CCB100274FF0D1
:1028F000010A09EB4712D2F8003B03F44023B3F579
:10290000802F11D1D2F8003B002B0DDA62890AFA30
:1029100007F322EA0303638104EB8703DB68DB68C8
:1029200013B1394658469847A36D01379B68FFB2EB
:102930009F42DED9E80617D5676D3A6AC2F30A10DE
:1029400002F00F0302F4F012B2F5802F00F088803D
:10295000B2F5402F08D104EB83030022DB681B6A29
:1029600007F5805790426DD12903D6F8184813D542
:10297000E20302D50020FFF795FEA30302D5012054
:10298000FFF790FE670302D50220FFF78BFE2603B8
:1029900002D50320FFF786FE6D037FF567AFE007E2
:1029A00002D50020FFF712FFA10702D50120FFF793
:1029B0000DFF620702D50220FFF708FF23077FF50E
:1029C00055AF0320FFF702FF50E7636DDFF8E8B073
:1029D000019300274FF0010AA36D9B685FFA87F906
:1029E00099453FF67DAF019B03EB4913D3F80029CE
:1029F00002F44022B2F5802F22D1D3F80029002A18
:102A00001EDAD3F8002942F09042C3F80029D3F827
:102A10000029002AFBDB606D4946FFF769FC22892B
:102A20000AFA09F322EA0303238104EB8903DB6832
:102A30009B6813B14946584698474846FFF71AFC29
:102A40000137C9E7910708BFD7F80080072A98BF68
:102A500003F8018B02F1010298BF4FEA182881E7C1
:102A6000023304EB830207F580575268D2F818C08E
:102A7000DCF80820DCE9001CA1EB0C0C00218842EA
:102A80000AD104EB830463689B699A6802449A60E4
:102A90005A6802445A6067E711F0030F08BFD7F87D
:102AA00000808C4588BF02F8018B01F1010188BFCD
:102AB0004FEA1828E3E700BFB02C0020436D03EB7A
:102AC0004111D1F8003B43F40013C1F8003B7047BB
:102AD000436D03EB4111D1F8003943F40013C1F801
:102AE00000397047436D03EB4111D1F8003B23F4EB
:102AF0000013C1F8003B7047436D03EB4111D1F85F
:102B0000003923F40013C1F80039704700F1604325
:102B100003F561430901C9B283F80013012200F0F3
:102B20001F039A4043099B0003F1604303F561438F
:102B3000C3F880211A60704730B5039C01720433DA
:102B400004FB0325C0E90653049B03630021059B96
:102B5000C160C0E90000C0E90422C0E90842C0E940
:102B60000A11436330BD0000416A0022C0E904112C
:102B7000C0E90A22C2606FF00101FEF705BF000044
:102B8000D0E90432934201D1C2680AB9181D7047D6
:102B90000020704703691960C2680132C260C269CF
:102BA000134482690361934224BF436A0361002195
:102BB000FEF7DEBE38B504460D46E3683BB16269F8
:102BC000131D1268A3621344E362002007E0237A16
:102BD00033B929462046FEF7BBFE0028EDDA38BDA2
:102BE0006FF00100FBE70000C368C269013BC360EE
:102BF0004369134482694361934224BF436A43613A
:102C000000238362036B03B11847704770B520231C
:102C1000044683F31188866A3EB9FFF7CBFF054669
:102C200018B186F31188284670BDA36AE26A13F8CA
:102C3000015BA362934202D32046FFF7D5FF002336
:102C400083F31188EFE700002DE9F84F04460E46A4
:102C5000174698464FF0200989F311880025AA46A7
:102C6000D4F828B0BBF1000F09D141462046FFF748
:102C7000A1FF20B18BF311882846BDE8F88FD4E975
:102C80000A12A7EB050B521A934528BF9346BBF1D6
:102C9000400F1BD9334601F1400251F8040B43F8B1
:102CA000040B9142F9D1A36A40334036A362403508
:102CB000D4E90A239A4202D32046FFF795FF8AF30C
:102CC0001188BD42D8D289F31188C9E730465A46E7
:102CD000FDF7D0FFA36A5B445E44A3625D44E7E76F
:102CE00010B5029C0172043304FB0321C0E90613F2
:102CF0000023C0E90A33039B0363049BC460C0E95B
:102D00000000C0E90422C0E90842436310BD00008E
:102D1000026AC260426AC0E904220022C0E90A22B3
:102D20006FF00101FEF730BED0E904239A4201D1D1
:102D3000C26822B9184650F8043B0B607047002067
:102D400070470000C368C2690133C360436913441C
:102D500082694361934224BF436A43610021FEF7C5
:102D600007BE000038B504460D46E3683BB1236951
:102D70001A1DA262E2691344E362002007E0237A8D
:102D800033B929462046FEF7E3FD0028EDDA38BDC9
:102D90006FF00100FBE7000003691960C268013AA7
:102DA000C260C269134482690361934224BF436ACB
:102DB000036100238362036B03B11847704700006F
:102DC00070B520230D460446114683F31188866AA8
:102DD0002EB9FFF7C7FF10B186F3118870BDA36A43
:102DE0001D70A36AE26A01339342A36204D3E169CE
:102DF00020460439FFF7D0FF002080F31188EDE76B
:102E00002DE9F84F04460D46904699464FF0200AAA
:102E10008AF311880026B346A76A4FB9494620466F
:102E2000FFF7A0FF20B187F311883046BDE8F88F87
:102E3000D4E90A073A1AA8EB0607974228BF1746B3
:102E4000402F1BD905F1400355F8042B40F8042B03
:102E50009D42F9D1A36A4033A3624036D4E90A23E4
:102E60009A4204D3E16920460439FFF795FF8BF3BA
:102E700011884645D9D28AF31188CDE729463A46CA
:102E8000FDF7F8FEA36A3B443D44A3623E44E5E7F8
:102E9000D0E904239A4217D1C3689BB1836A8BB1EE
:102EA000043B9B1A0ED01360C368013BC360C36927
:102EB0001A44836902619A4224BF436A0361002372
:102EC00083620123184670470023FBE700F088B8AF
:102ED0004FF08043002258631A610222DA60704783
:102EE0004FF080430022DA60704700004FF08043CB
:102EF000586370474FF08043586A70474B6843608F
:102F00008B688360CB68C3600B6943614B69036264
:102F10008B6943620B6803607047000008B5264B5D
:102F200026481A6940F2FF110A431A611A6922F40D
:102F3000FF7222F001021A611A691A6B0A431A63BE
:102F40001A6D0A431A651E4A1B6D1146FFF7D6FF1C
:102F500002F11C0100F58060FFF7D0FF02F138019B
:102F600000F58060FFF7CAFF02F1540100F58060B0
:102F7000FFF7C4FF02F1700100F58060FFF7BEFFAC
:102F800002F18C0100F58060FFF7B8FF02F1A801A3
:102F900000F58060FFF7B2FF02F1C40100F5806028
:102FA000FFF7ACFF02F1E00100F58060FFF7A6FF3C
:102FB000BDE8084000F09AB8003802400000024026
:102FC0006836000808B500F007FAFEF731FCFFF795
:102FD0008DF8BDE80840FEF753BE000070470000C2
:102FE000104B1A6C42F001021A641A6E42F0010290
:102FF0001A660D4A1B6E936843F0010393604FF00D
:10300000804353229A624FF0FF32DA6200229A61C3
:103010005A63DA605A6001225A6108211A601C2042
:10302000FFF774BD00380240002004E04FF08042FA
:1030300008B51169D3680B40D9B2C9439B07116128
:1030400007D5202383F31188FEF712FC002383F3B6
:10305000118808BD08B5FFF7E9FFBDE80840FFF794
:103060008FB800001F4B1A696FEAC2526FEAD25242
:103070001A611A69C2F308021A614FF0FF301A6927
:103080005A69586100215A6959615A691A6A62F08D
:1030900080521A621A6A02F080521A621A6A5A6AD6
:1030A00058625A6A59625A6A1A6C42F080521A641B
:1030B0001A6E42F080521A661A6E0B4A106840F47B
:1030C00080701060186F00F44070B0F5007F1EBF74
:1030D0004FF4803018671967536823F40073536006
:1030E00000F05AB90038024000700040334B4FF0F6
:1030F00080521A64324A4FF4404111601A6842F01B
:1031000001021A601A689107FCD59A6822F003023E
:103110009A602A4B9A6812F00C02FBD1196801F0F0
:10312000F90119609A601A6842F480321A601A68CC
:103130009203FCD55A6F42F001025A671F4B5A6F37
:103140009007FCD51F4A5A601A6842F080721A60D4
:103150001B4A53685904FCD5184B1A689201FCD5D8
:10316000194A9A60194B1A68194B9A42194B21D186
:10317000194A1168194A91421CD140F205121A608D
:10318000144A136803F00F03052BFAD10B4B9A680E
:1031900042F002029A609A6802F00C02082AFAD100
:1031A0005A6C42F480425A645A6E42F480425A6623
:1031B0005B6E704740F20572E1E700BF00380240E5
:1031C000007000400854400700948838002004E054
:1031D00011640020003C024000ED00E041C20F41BC
:1031E000084A08B5516913680B4003F001035361A5
:1031F00023B1054A13680BB150689847BDE80840F1
:10320000FEF7BEBF003C0140282D0020084A08B54B
:10321000516913680B4003F00203536123B1054A5F
:1032200093680BB1D0689847BDE80840FEF7A8BF87
:10323000003C0140282D0020084A08B55169136858
:103240000B4003F00403536123B1054A13690BB12A
:1032500050699847BDE80840FEF792BF003C014026
:10326000282D0020084A08B5516913680B4003F067
:103270000803536123B1054A93690BB1D06998479C
:10328000BDE80840FEF77CBF003C0140282D00202F
:10329000084A08B5516913680B4003F010035361E5
:1032A00023B1054A136A0BB1506A9847BDE808403C
:1032B000FEF766BF003C0140282D0020174B10B5DB
:1032C0005A691C68144004F478725A61A30604D544
:1032D000134A936A0BB1D06A9847600604D5104A26
:1032E000136B0BB1506B9847210604D50C4A936BB6
:1032F0000BB1D06B9847E20504D5094A136C0BB1AA
:10330000506C9847A30504D5054A936C0BB1D06C5B
:103310009847BDE81040FEF733BF00BF003C0140B6
:10332000282D00201A4B10B55A691C68144004F46B
:103330007C425A61620504D5164A136D0BB1506D7B
:103340009847230504D5134A936D0BB1D06D984768
:10335000E00404D50F4A136E0BB1506E9847A104D8
:1033600004D50C4A936E0BB1D06E9847620404D515
:10337000084A136F0BB1506F9847230404D5054AD0
:10338000936F0BB1D06F9847BDE81040FEF7F8BEC1
:10339000003C0140282D0020062108B50846FFF713
:1033A000B5FB06210720FFF7B1FB06210820FFF738
:1033B000ADFB06210920FFF7A9FB06210A20FFF734
:1033C000A5FB06211720FFF7A1FBBDE80840062159
:1033D0002820FFF79BBB000008B5FFF743FE00F075
:1033E0000BF8FDF7E3FEFDF7BBFDFFF7F7FDBDE8CA
:1033F0000840FFF76BBD00000023054A1946013362
:10340000102BC2E9001102F10802F8D1704700BF89
:10341000282D0020034611F8012B03F8012B002A68
:10342000F9D1704753544D3332463F3F3F000000BF
:1034300053544D3332463430780053544D33324672
:103440003432780053544D333246343436585800B1
:10345000012033000010410001105A0003105900F0
:103460000710310000000000243400083F00000075
:1034700013040000303400083F000000190400006D
:103480003A3400083F0000002104000044340008E2
:103490003F00000000000000DD0E0008C90E00081B
:1034A000050F0008F10E0008FD0E0008E90E0008E7
:1034B000D50E0008C10E0008110F00080000000022
:1034C00001000000000000006D61696E0000000056
:1034D00069646C6500000000D0340008D823002027
:1034E00050250020010000002D18000800000000F9
:1034F0004172647550696C6F740025424F415244AB
:10350000252D424C002553455249414C25000000D1
:103510000200000000000000F9100008651100081A
:1035200040004000E8290020F829002002000000A7
:10353000000000000300000000000000A9110008C6
:103540000000000010000000082A00200000000019
:103550000100000000000000B02C0020010102006A
:103560001D1C00082D1B0008C91B0008AD1B00080E
:10357000430000007835000809024300020100C042
:1035800032090400000102020100052400100105B7
:10359000240100010424020205240600010705821B
:1035A000030800FF09040100020A000000070501EA
:1035B00002400000070581024000000012000000E8
:1035C000C4350008120110010200004009124157E1
:1035D00000020102030100000403090425424F41D7
:1035E00052442500466C79776F6F46343035532D41
:1035F00041494F0030313233343536373839414262
:103600004344454600000000004000000040000028
:103610000040000000400000000001000000020027
:103620000000020000000200000002000000020092
:10363000000002000000020000000000E11200088B
:10364000991500084516000840004000102D002084
:10365000102D002001000000202D0020800000001F
:1036600040010000030000000000842A0000000068
:10367000AAAAAAAA00000024FFFD00000000000082
:1036800000A00A004000001100000000AAAAAAAA97
:1036900040000011FFFF00000000000000000000DB
:1036A0000000000000000000AAAAAAAA0000000072
:1036B000FFFF00000000000000000000000000000C
:1036C00000000000AAAAAAAA00000000FFFF000054
:1036D00000000000000000000000000000000000EA
:1036E000AAAAAAAA00000000FFFF00000000000034
:1036F000000000000000000000000000AAAAAAAA22
:1037000000000000FFFF00000000000000000000BB
:103710000000000000000000AAAAAAAA0000000001
:10372000FFFF00000000000000000000000000009B
:10373000000000000A00000000000000030000007C
:103740000000000000000000000000000000000079
:103750000000000000000000000000000000000069
:1037600000000000000000004B040000000000000A
:1037700000400F0000000000FF009600000000085D
:10378000009600000000080004000000D835000882
:103790000000000000000000000000000000000029
:0837A000000000000000000021
:00000001FF
